:100000000C94A2050C94CB050C94CB050C94CB0559
:100010000C94CB050C94CB050C94CB050C94500D93
:100020000C94CB050C94CB050C94CB050C94CB0510
:100030000C94CB050C94CB050C94CB050C94CB0500
:100040000C94CB050C94CB050C94CB050C94CB05F0
:100050000C94CB050C94CB050C94CB050C94CB05E0
:100060000C94CB050C94CB05D710D710D710D71014
:10007000D710D710D710D710D710D710D710D71048
:10008000D710D710D710D710D71077107A10D710F5
:100090007F108310871087108710871087108710B4
:1000A000D510951099109910991099109910D51094
:1000B000A610AA10AA10AA10AA10AA10D710D7101A
:1000C000D710B710B910B910B910B910C610C810B0
:1000D000C810C810C810C810C810C810D5104919C9
:1000E0004C194F195219551958195B195E19611994
:1000F000641967196A196D196F1A6F1A691A6F1ADC
:100100006C1A761A6F1A6F1A731A761A761A791A87
:10011000791AAB1AA81AA21AA51AB31AB31AA81AEE
:10012000AB1AB01AB31AB31AB31AB31ACB1AD31A3A
:10013000DD1AE51AED1AF51AFD1A051B0D1B151B24
:100140001D1B251B291BAC1BAF1BB41BB71BBA1BEC
:10015000BD1BC01BC31BC61BC91BCC1B0204010457
:10016000020403060406020400060005000500055B
:100170000005000500060300050103060406050648
:100180000006010602060306040602030006010635
:100190000206050105010506000601060206050125
:1001A000040605060006010602060402040605060A
:1001B0000006010602060306030005060006020605
:1001C00002060306040605060006010601060306EC
:1001D00004060506010001020104000502030205F0
:1001E00000050105000140400060003000180808CB
:1001F0000C00060042002D2D2000202D2D00204F48
:1002000063744574372000031014000310111400A8
:1002100000000013000000000000000000000010BB
:100220000000001300000000000000101400001087
:100230001400001011140013150000031300000037
:100240000000001300000002090A0B0C0D0E0F1233
:1002500018190000006501610078027801780065D6
:1002600007780278037804780065037805780065DC
:1002700004780678006505780B3000650678087804
:10028000077800650065087809780A7800650978BC
:100290000B3100650A780C7801610B780065016DFF
:1002A0000C7800000000000000000000000000FFCB
:1002B0000100000040DB40CF40C340B840AE40A446
:1002C000409B4092408A4082407B4074406D406732
:1002D0004061405C40564051404D404840444040A1
:1002E000403D4039403640334030402D402B40287F
:1002F000402640244022402008F608E808DB08CFCA
:1003000008C308B808AE08A4089B0892088A0882A7
:10031000087B0874086D08670861085C0856085176
:10032000084D084808440840083D08390836083395
:100330000830082D082B0828082608240822082041
:1003400001F601E801DBFF000003020500030501DF
:100350000406020472083008EE07B80776072B0778
:10036000DD068F06450558040D04C20300494949BE
:100370004949494949494949490149497E306D79C5
:10038000335B5F707F734949494949494977494E11
:10039000494F474937063C490E49497E6749495B01
:1003A000493E4949494949494949490849491F0D6F
:1003B0003D494949170449494949151D49490549D4
:1003C0000F1C03300004060A03060004300A030071
:1003D0000004000002300005060A02060005300A8B
:1003E00002000005000001300006060A01060006B2
:1003F000300A01000006000000300007060A00066F
:100400000007300A000000070000FF0000FD0000A8
:10041000000603007E03004E00010603017803017D
:10042000480002060302780302480003060303782B
:100430000303480004060304780304480005060388
:1004400005780305480006060306780306480007FA
:100450000603077832FF000003300004060A030792
:100460000004310A03010004010002300005060AFD
:1004700002060005300A02000005000001300006F7
:10048000060A01070006310A0101000601000030DA
:100490000007060A00070007310A000100070132C1
:1004A00000200001040003200004040006200007CF
:1004B00004090010000102000310000402000610ED
:1004C000000702090001000101000301000401000E
:1004D00006010007010900200001040003200004B8
:1004E00004000620000704090010000102000310A8
:1004F00000040200061000070209000100010100CB
:1005000003010004010006010007010900200001A9
:100510000400032000040400062000070409001062
:100520000001020003100004020006100007020987
:1005300000010001010003010004010006010007A1
:100540000150FF0000FD000000020007100A00201B
:100550000007040500000007000001020006100269
:10056000012000060401010000060000020200054F
:100570001001022000050401020000050000030232
:100580000004100103200004040103000004000023
:10059000040200031001042000030401040000030E
:1005A0000000050200021001052000020401050000
:1005B00000020000060200011001062000010402F2
:1005C00006000001000007020000100507200000DF
:1005D00004050002000710050020000704050000C4
:1005E00000070000010200061002012000060401BD
:1005F00001000006000002020005100102200005B3
:1006000004010200000500000302000410010320A1
:1006100000040401030000040000040200031001B0
:10062000042000030401040000030000050200028E
:10063000100105200002040105000002000006026E
:100640000001100106200001040206000001000064
:100650000702000010030720000004040008000146
:10066000000500180001080500110001180500032D
:1006700000013005004200016005006200014205F2
:10068000006300010605007700010E05FF0000FD74
:100690000000000105010105020105030105033108
:1006A00005057700063E00075B1405000006000004
:1006B000070014057700063E00075B1405000006DE
:1006C0000000070014057700063E00075B5000009D
:1006D00005010005020005030005FF0000FD000004
:1006E00000010501010502010503010503310505AE
:1006F0004F0006040007151405000006000007005F
:1007000014054F000604000715140500000600003C
:10071000070014054F0006040007155000000501EE
:100720000005020005030005FF0000033000040679
:100730000A03060004300A0300000400000230002F
:1007400005060A02060005300A0200000500000145
:10075000300006060A01060006300A010000060005
:100760000000300007060A00060007300A000000FB
:10077000070000FF0000FD0000007700010E0004EC
:100780000000050000060014047700053E00065B2B
:1007900014040000050000060014047700053E0064
:1007A000065B140400000500000600140477000531
:1007B0003E00065BC8FF0000FD00000006090001C6
:1007C00009010109020109030109040109050109DF
:1007D000050000067700070E190000090100090254
:1007E0000009030009040009050009FF0000FD00DD
:1007F00000007700010E0004000005000006001450
:10080000047700053E00065B1404000005000006A6
:100810000014047700053E00065B14040000050088
:1008200000060014047700053E00065BC8FF0000C8
:10083000FD0000007700010E000400000500000626
:100840000014044F00050400061514040000050000
:1008500000060014044F00050400061514040000EF
:10086000050000060014044F000504000615C8FF2B
:100870000000000109010109020109020000030151
:1008800009040109050109050000060109070132F3
:1008900000200001040003200004040006200007DB
:1008A00004090010000102000310000402000610F9
:1008B000000702090001000101000301000401001A
:1008C00006010007010900200001040003200004C4
:1008D00004000620000704090010000102000310B4
:1008E00000040200061000070209000100010100D7
:1008F00003010004010006010007010900200001B6
:10090000040003200004040006200007040900106E
:100910000001020003100004020006100007020993
:1009200000010001010003010004010006010007AD
:10093000015AFF00002D2D202D2D00414C20202D8F
:100940002D2D2000414C202045696E2000414C2077
:10095000204155532000414C20000080C0E0F0F8B9
:10096000FCFEFF2D2D2D002D2D004A41004C303175
:10097000004C3032004C3033004C3034004C3035B9
:10098000004C3036004C3037004C3038004C303999
:10099000004C3130004C3131004C3132004C31339D
:1009A000004C3134004C3135004C31360041555348
:1009B0000045696E00536F756E6400724164696F23
:1009C00000312D74202000322D74452000332D7409
:1009D000454600342D45202000352D454620003663
:1009E0002D46202000372D45696E002D2D005374B3
:1009F0004172740072455345740064537400416E33
:100A00004672004C416E6400536E6F4C4500536E4D
:100A10006F53456E00536E6F6F00417400414C453B
:100A20006E00414F004C456453456E004C454155A6
:100A300053002A0BF00AE80AE40ADC0AD60ACE0AB6
:100A4000C80AC00AB80AB20AA00A9C0A8C0A800A1C
:100A5000720A620A5E0A580A1905310F0000311441
:100A60000000310A00142C08000329080003250A9D
:100A70000000250A000A29062C062E06310F000068
:100A8000250A000820081D08190F00003D0200502B
:100A90003D0200503D0200503D020000250A0000CA
:100AA000310A2C0A2A0A2C0A310A0046193200C8D7
:100AB0004A01190A25140000310A00022514000019
:100AC000250A0002311400003105250A000019052D
:100AD0002502310A00003D0525140000250700010C
:100AE0003D0A00003D010000250700143D280000DC
:100AF00001010004010100040101000401010004DE
:100B000001010004010100040101000401010004CD
:100B100001010004010100040101000401010004BD
:100B200001010004010100040000250529052C0530
:100B3000310F000005050000140700000001050545
:100B40000901010011241FBECFEFD8E0DEBFCDBFE9
:100B500014BE0FB6F894A8958091600088618093C8
:100B60006000109260000FBE11E0A0E0B1E0EEE581
:100B7000FCE302C005900D92A038B107D9F721E03F
:100B8000A0E8B1E001C01D92AA3BB207E1F70E94C4
:100B900060170C942D1E0C940000FF920F931F936E
:100BA000CF93DF93CDB7DEB72E970FB6F894DEBFA5
:100BB0000FBECDBF182FCE0101960E94280FCE0187
:100BC00001960E941D15882309F480C041E050E081
:100BD000BE01625F7F4F8EE090E00E94091CAE0173
:100BE0004F5F5F4F6E8581E00E94B31589819A81C6
:100BF000AB818B879C87AD8743E050E0BE01685F87
:100C00007F4F85E090E00E94091CCE0108960E946B
:100C10003F12882309F45AC088859985AA8589835B
:100C20009A83AB83BE01655F7F4FCE0108960E9419
:100C3000501218162CF061E0CE0104960E94231386
:100C4000FF24F394CE0104960E9459130AEF080F73
:100C5000CE0104960E94AF130E94EE081330A1F05B
:100C600028F4113049F0123051F020C0143079F0DE
:100C70001530E1F48F2512C0023090F017C0023019
:100C800060F481E090E009C0023050F40FC00230FF
:100C900010F08F2502C080E090E08170882331F051
:100CA00061E0CE0101960E945915CCCFAE014F5F95
:100CB0005F4F6E8581E00E94CF1587E0FE0131967F
:100CC000ACE0B1E001900D928A95E1F72E960FB657
:100CD000F894DEBF0FBECDBFDF91CF911F910F9172
:100CE000FF9008950F931F93CF93DF93CDB7DEB797
:100CF00027970FB6F894DEBF0FBECDBF8C01CE0193
:100D000001960E94280FCE0101960E941D1588238E
:100D1000E1F0F8016081CE0101960E942F15F801E3
:100D20006181CE0101960E943D15F8016281CE01DC
:100D300001960E944B156CE071E0CE0101960E9475
:100D40005C158095881F8827881F27960FB6F89412
:100D5000DEBF0FBECDBFDF91CF911F910F910895E0
:100D6000882319F010921301089581E080931301F4
:100D7000089580918101811107C081E09091130154
:100D8000992319F080E001C081E08170089590916D
:100D90008101915081E0923008F080E008959091B7
:100DA0008101935081E0923008F080E0089581E065
:100DB00090918101943009F080E00895CF93DF9302
:100DC00000D01F92CDB7DEB719821A828FE08B83D5
:100DD00080918101882329F0CE0101960E9472063C
:100DE00001C080E00F900F900F90DF91CF91089598
:100DF0000F931F93CF93DF93CDB7DEB729970FB62D
:100E0000F894DEBF0FBECDBF41E050E0BE01675F8A
:100E10007F4F88E090E00E94091C80911301882395
:100E200029F0813031F402E010E005C001E010E06B
:100E300002C000E010E082E08093130119821A8260
:100E40001B8280918101882331F0CE0101960E949E
:100E50007206811104608BE089831A821B82809163
:100E60008101882331F0CE0101960E947206811122
:100E70000860809181018350823020F40E94D40860
:100E80008111006188E091E00E94261981110062C1
:100E900041E050E0BE01685F7F4F89E090E00E9432
:100EA000091C8885882389F184E091E00E942E192D
:100EB000882359F10E94640F882301F141E050E03A
:100EC000BE016F5F7F4F81E090E00E94091C998115
:100ED00089E0891B898320918001422F022E000C1A
:100EE000550B38E08302C00111244817590724F438
:100EF0002F5F2093800109C0006407C080918001AA
:100F000018161CF481508093800180E091E00E94CB
:100F10002619811100680E94C808813009F011600B
:100F20008985882321F00E94E208811111600E94C6
:100F3000C808813049F48985811102C0126004C05B
:100F40000E94E2088823D1F360918101862F90E00E
:100F5000880F991F845A9E4F20E030E0A1E0B0E056
:100F6000AD01022E02C0440F551F0A94E2F7402340
:100F70005123452BE1F0FC0144913196E491641733
:100F8000A1F040938101E23009F45CC028F4EE2323
:100F9000A9F0E130B9F1ACC0E43009F486C008F43E
:100FA0007DC0E53009F490C0A3C0E63051F72F5F53
:100FB0003F4F0C962A30310599F69EC089858823CB
:100FC00029F081E00E948A0F8AE001C08BE00E9434
:100FD000FB1B41E050E0BE016F5F7F4F84E090E07B
:100FE0000E94091C6981FCE36F9FB001112488E015
:100FF00091E00E94ED1883E00E94481783E00E9470
:101000008C1678C08985882349F00E94E2088111F6
:1010100005C00E948A0F80E00E94490F84E00E9470
:10102000481780E00E948C168EE00E94FB1B41E076
:1010300050E0BE016F5F7F4F83E090E00E94091C8B
:1010400089813FC08985882331F080E00E948A0F22
:1010500080E00E94490F41E050E0BE01685F7F4F91
:101060008BE090E00E94091C08853CE3039F80010F
:101070001124CE0101960E94280F8B81853110F436
:10108000081B1109B80180E091E00E94ED1880E092
:101090000E948C168CE00E94FB1B2CC08DE00E94ED
:1010A000FB1B81E00E94481725C081E0898341E055
:1010B00050E0BE016F5F7F4F82E090E00E940C1C09
:1010C00080E00E94CD0516C00E94E208811105C093
:1010D0000E948A0F80E00E94490F198241E050E08F
:1010E000BE016F5F7F4F82E090E00E940C1C02C047
:1010F000E63011F00E94EA0829960FB6F894DEBF98
:101100000FBECDBFDF91CF911F910F9108950F9327
:101110001F93CF93DF931F92CDB7DEB78C010E9450
:10112000280F41E050E0BE016F5F7F4F8EE090E0FE
:101130000E94091CA801698181E00E94B3150F90EB
:10114000DF91CF911F910F9108956230E8F0E7E4AD
:10115000F2E094916917D1F0319622E0E235F2077E
:10116000C1F724E0829FC001112420E030E0F901A2
:10117000E80FF91FE95FFD4FE4916E1739F02F5F1B
:101180003F4F2430310599F780E0089581E00895BC
:1011900080912F01089580932F01089580918701F8
:1011A000089580918601089580918701811107C07B
:1011B00081E090918601911103C080E001C081E03F
:1011C0008170089590918801915081E0923008F0EB
:1011D00080E0089581E080932E0108951F93CF93BE
:1011E000DF931F92CDB7DEB7182F41E050E0BE016C
:1011F0006F5F7F4F8CE090E00E94091C612F898116
:101200000E94A5080F90DF91CF911F9108950F9331
:101210001F93CF938C010E945913C82FC8010E94BD
:10122000AF130E94EE08C650C23010F481E090E087
:101230008170CF911F910F910895CF938EEF91E020
:101240000E945C1680E00E94FB1BC0E08AE291E0F5
:101250000E942E19882319F08C2F0E94EF158AE224
:1012600091E00E942619811105C00E94EF0F0E9493
:10127000A116F5CFCF5FCE3149F710922F01CF9154
:101280000895FF920F931F93CF93DF93CDB7DEB7EF
:1012900061970FB6F894DEBF0FBECDBF0E948916CE
:1012A0008C3009F00AC18091290190912F01891792
:1012B000B9F0913051F038F0923059F0933059F440
:1012C0000E94131A08C082E401C080E00E948C16BC
:1012D00002C00E947D1780912F0180932901EDC0EB
:1012E000813009F45EC048F0823009F4E4C08330F4
:1012F00009F0E3C00E943C1AE0C0CE010B960E94A8
:101300008708CE010B960E941D158E010F5F1F4F9F
:101310008823B9F080E00E94481781E00E94FB1BFF
:1013200041E050E0B80182E090E00E94091C898110
:10133000882319F081E00E94B00681E080932F019C
:101340002AC08AE0F80111928A95E9F76AEF71E004
:10135000C8010E945D1D0E943E0FFC01F080F9E073
:10136000FF1520F060E3C8010E943D1D6F2D70E065
:10137000C8010E94711D66EF71E0C8010E945D1DE9
:10138000C8010E943C1661E382E00E94041667E0F7
:1013900085E00E9404160E94740F893208F081C013
:1013A0008CC0CE010B960E948708CE010B960E943E
:1013B0001D15882309F46BC08E010F5F1F4F8AE053
:1013C000F80111928A95E9F78B858A3020F460E262
:1013D000C8010E943D1D6B8570E0C8010E94711D0F
:1013E0006DE2C8010E943D1D8C858A3020F460E3C7
:1013F000C8010E943D1D6C8570E0C8010E94711DEE
:101400000E94CF06882379F160E2C8010E943D1D49
:101410000E94D7068823B9F185E291E00E942E1937
:10142000882389F1E0918501F0E0EE0FFF1FEA517A
:10143000FE4F649186E00E940416E0918501F0E081
:10144000EE0FFF1FE951FE4F649187E00E940416E2
:10145000809185018F5F883019F08093850113C0DA
:101460001092850110C06DE2C8010E943D1D8D855E
:101470008A3020F460E3C8010E943D1D6D8570E054
:10148000C8010E94711DC8010E943C1602C0109242
:101490002F010E94CF06811110C00E94740F893263
:1014A00010F083E005C080918601882331F082E04E
:1014B00080932F0102C00E9494170E94680F8093AE
:1014C00087010E947E0F8093860190918701911180
:1014D00002C0882319F081E080932E01809184015D
:1014E000882341F00E9489168C3021F410928701E4
:1014F000109286010E94891691E08C3009F490E0E8
:101500009093840181E291E00E942E19882369F171
:101510000E94640F882311F141E050E0BE016F5F2B
:101520007F4F81E090E00E94091C998189E0891B2E
:10153000898320918301422F022E000C550BF8E085
:101540008F02C00111244817590724F42F5F2093FC
:1015500083010BC081E080932E0107C0809183013D
:1015600018161CF481508093830110912F010E9462
:10157000DE06811107C08EEF810F11E0823018F076
:1015800010E001C011E080912E01811111E0109254
:101590002E018DE191E00E942619811112600E94B6
:1015A0008916853009F0146060918201262F30E0A1
:1015B000220F331F2C523E4F40E050E0812F90E02D
:1015C000FC01042E02C0F595E7950A94E2F7E0FFCE
:1015D0002DC0F90174913196E491671729F1709348
:1015E0008201E230E9F148F4EE2341F1E13009F003
:1015F0004EC080E00E94E5154AC0E33009F43FC0C8
:10160000E43009F044C00E94821641E050E0BE017F
:101610006F5F7F4F80E090E00E94091C69813CE38E
:10162000639FB00111242FC0E530C9F64F5F5F4FB3
:101630002A5F3F4F4330510551F1C2CF81E00E94F4
:10164000E51541E050E0BE016F5F7F4F80E090E024
:101650000E94091C6981FCE36F9FB001112413C033
:1016600041E050E0BE016F5F7F4F80E090E00E945C
:10167000091C69812CE3629FB001112404C085E03C
:101680000E94481704C08DE191E00E94ED188091FE
:101690002F018130F9F489E191E00E942E1988230D
:1016A00001F10E94460F87FD84E6E4E68E02C00148
:1016B0001124835B9E4F6AE972E00E94E11D162FA0
:1016C0000E940116181714F4815009C081174CF4B8
:1016D0008F5F05C00E9401168F3019F08FE00E94C5
:1016E000EF150E94CF06882321F00E94F50E81702D
:1016F00002C00E94C706682F83E00E941C160E9449
:10170000410F882321F00E94E70E692F11C00E942B
:101710003E0FFC01818192818438934058F00E94F1
:10172000E70E8078927061E08038910509F060E002
:10173000617001C060E084E00E941C1641E050E04E
:10174000BE01655F7F4F8DE090E00E94091C8B8594
:10175000882349F0CE0101960E948708CE010496A5
:101760000E94070901C080E0682F87E00E941C16D4
:101770000E94CF06882331F00E94F50E80FF5AC0E8
:1017800084E659C0809187018823B1F080912F01B0
:10179000823090F40E9489168C3071F48091880117
:1017A000811103C081E0809388018091880182309B
:1017B00019F483E08093880110918801123099F028
:1017C000133061F1113099F586E00E94FB1B86E031
:1017D0000E94481780E00E94490F1093180182E090
:1017E000809388012AC081E00E948A0F84E191E001
:1017F0000E942E19882309F10E94610F909118010F
:10180000992331F08F5F8436B1F41092180113C020
:10181000815089F491E0909318010DC087E00E94F7
:10182000FB1B87E00E9448171092880106C080E0E9
:101830000E948A0F80E00E94490FCE0101960E940B
:101840008708CE0104960E9407090E94900F0E940B
:10185000CF060E94960F0E94F80661960FB6F89484
:10186000DEBF0FBECDBFDF91CF911F910F91FF90D3
:101870000895089587E090E001970000E9F7089542
:1018800087FF01C078940895CF93DF93EC010E9405
:101890001D15882369F08FB7F89497E0FE01A2E444
:1018A000B1E001900D929A95E1F710929B0105C06D
:1018B0008FB7F8949FEF90934401DF91CF910C94F0
:1018C000400CEF92FF920F931F93CF93DF93E82E7C
:1018D000D92FF62E84EA8093BC00C4E68091BC0028
:1018E00087FD07C0CC2309F442C00E943A0CC150C6
:1018F000F5CFCC23E1F18091B900887F8830B9F52C
:1019000080ED8093BB0084E88093BC00C4E68091A6
:10191000BC0087FD06C0CC2351F10E943A0CC15097
:10192000F6CFCC2321F18091B900887F8831F9F47A
:101930000E2D1D2FC0E084E8E82E06C08091B9006E
:10194000887F883289F4CF5FCF1571F0F8018191DB
:101950008F018093BB00E092BC00D4E68091BC0074
:1019600087FF07C0D111EACF81E0FC1641F080E08B
:1019700006C0DD23C9F30E943A0CD150EFCF94E9A1
:101980009093BC00E9E4F0E031970000E9F7109291
:10199000BC00DF91CF911F910F91FF90EF900895C0
:1019A000FF920F931F93CF93DF93CDB7DEB72997A5
:1019B0000FB6F894DEBF0FBECDBF8C0119820E9416
:1019C0001D15882309F455C0D80112968C919AE010
:1019D000F92E6F2D0E94C11DB0E18B9F900D112437
:1019E0009A83F80181810E94C11DF0E18F9F900DC3
:1019F00011249B83D8018C910E94C11DB0E18B9F63
:101A0000900D11249C83C80103960E9459138D8365
:101A1000F80183816F2D0E94C11DF0E18F9F900D11
:101A200011249E83D80114968C910E94C11DB0E1AF
:101A30008B9F900D11249F83D8011596ED91FC91F9
:101A40001697CF0164E670E00E94CD1D2AE030E0D9
:101A5000B9010E94CD1D462FCF01B9010E94CD1DB5
:101A6000B0E14B9F800D1124888780E1898769E070
:101A700003C080E88A8362E0CE0101960E94610C77
:101A8000809398018091980129960FB6F894DEBF53
:101A90000FBECDBFDF91CF911F910F91FF900895A1
:101AA0001F920F920FB60F9211242F933F934F93D3
:101AB0005F936F937F938F939F93AF93BF93CF93D6
:101AC000DF93EF93FF9380919701843021F410927C
:101AD000970183E704C08F5F8093970182E780932B
:101AE000B300C0919601CF5FCA3029F0C093960130
:101AF00080E0D0E019C010929601809195018F5F2F
:101B00008A3019F080939501F3CF1092950180915E
:101B100094018F5F8A3021F08093940180E003C0AC
:101B20001092940181E0D1E02091A5013091A601AD
:101B30002F5F3F4F3093A6012093A501882349F0E2
:101B40008091A3019091A40101969093A4018093A8
:101B5000A301CA30A1F480919B018F5F80939B0108
:101B600080919B01843659F410929B01809144012D
:101B70008C3328F461E082E491E00E944B154A9B8B
:101B800002C080E001C082E099B193FB992790F9EF
:101B900021E09227980F80919301E92FF0E024E053
:101BA000829FE00DF11D1124EE55FD4FE4918091CF
:101BB0009201E80FE0939201909393018091A0012C
:101BC000E13021F48F3728F48F5F03C0EF3F19F421
:101BD0008150109292018093A001CA3059F589B1C9
:101BE000807190919101992361F0882331F0909157
:101BF0009001992311F0915001C095E090939001CC
:101C00000DC0811106C090919001992311F091505F
:101C100001C092E0909390011092A10190919001E7
:101C20009111BBC091E0811190E09093910190934C
:101C3000A201B3C0DD2309F4B4C0809191018823CF
:101C400049F08091A1018A3F28F48091A1018F5F22
:101C50008093A101CA3009F0A4C080919F0188231C
:101C600009F45AC080919F01815080939F01809117
:101C70009F01811151C020919E0180919E018F5F33
:101C800080939E01E0919C01F0919D0130E0220F34
:101C9000331FE20FF31F8491E0919C01F0919D01AD
:101CA000E20FF31F3196249110928100109285006B
:101CB0001092840090E0880F991FFC01EE54FD4FB4
:101CC0003491FC01ED54FD4F849190E09093890094
:101CD00080938800383079F038F43130B9F480E4FA
:101CE0008093800089E00BC0303461F03F3F71F495
:101CF00010929E010BC080E4809380008AE0809364
:101D0000810008C0309380008BE0F9CF10928000F2
:101D10001092810020939F0180918F01863091F075
:101D20008F3081F0982F977F913161F08F3551F08E
:101D3000883741F08C3D31F0329902C022E003C077
:101D400021E001C020E080918E0190E0FC01EE0FC7
:101D5000FF1F8E0F9F1F820F911D880F991FFC017F
:101D6000EB5AFD4F2491FC01EC5AFD4F8491809376
:101D70008E012D3619F410928F0107C0213619F407
:101D800010928F0104C0283711F0209349018091EF
:101D90008F018F5F80938F0104C0DD2309F45DCF35
:101DA0004CCFFF91EF91DF91CF91BF91AF919F9178
:101DB0008F917F916F915F914F913F912F910F90F4
:101DC0000FBE0F901F901895109241010895CF9368
:101DD000DF938FB7F894C091A501D091A6010E941E
:101DE000400CCE01DF91CF910895CF93DF938FB751
:101DF000F894C091A301D091A4010E94400CCE019F
:101E0000DF91CF9108959C01CB01B9010C94FB1D8A
:101E10009C01CB01B9010C940B1E2A988EBD0DB408
:101E200007FEFDCF6EBD0DB407FEFDCF2A9A0895C3
:101E30009C018FB7F894ECE9F1E0318320831282A2
:101E400091E093830C94400C82E592E00C94180F7F
:101E5000DC018FB7F89497E0E2E4F1E001900D9295
:101E60009A95E1F70C94400CCF93DF93EC010E941C
:101E7000440CCE01DF91CF910C94D00C8EE391E015
:101E800008959091980181E08927089580919A01A1
:101E9000089587FD80E0282F85360CF024E6220285
:101EA000C001112467E270E00E94E11D611581E02C
:101EB000780719F48FEF87BD01C067BD20939901A2
:101EC000089580919901089586B18695817008954D
:101ED000CF938FB7F894C091A2011092A2010E94F3
:101EE000400C8C2FCF910895CF938FB7F894C09169
:101EF000A1010E94400C8C2FCF910895CF938FB7F2
:101F0000F894C091A0011092A0010E94400C8C2F67
:101F1000CF910895882311F0439A08954398089526
:101F2000882311F0589A089558980895882311F03D
:101F3000599A089559980895F8949FE088E10FB64A
:101F4000F894A895809360000FBE909360008FE393
:101F500084B994E095B988E087B918B883EE8AB956
:101F60001BB8E9E4F0E031970000E9F7EAE7F0E0B8
:101F700085E8808380818660808384B5816884BDA4
:101F800085B5836085BD17BCE0E8F0E080818064A2
:101F90008083E1E8F0E0808188608083109289008E
:101FA0001092880082E08093B00023E02093B1007B
:101FB00022E72093B3008093700080E58CBD81E020
:101FC0008DBD9093BC001092BA0084E68093B80057
:101FD0001092B90078940895809141010895BF92BC
:101FE000CF92DF92EF92FF920F931F93CF93DF93E5
:101FF000CDB7DEB765970FB6F894DEBF0FBECDBF85
:102000008AE391E00E942E19882369F080913F01B4
:102010009091400180362AEE920728F40196909321
:10202000400180933F018FB7F8941091490198E7E0
:10203000909349010E94400C80913E011D36C9F5E4
:102040008B3309F040C01B8280918D018A8380917F
:102050008C018983809139018C83809138018D8333
:1020600080918B0190E08053984F9F838E83CE01A7
:1020700001960E941D15882331F180918A018111FA
:1020800002C06FEF01C06EEFCE0101960E942F15C6
:10209000CE0101960E94440CCE0101960E94D00C04
:1020A0008AE391E00E94D2181092400110923F0101
:1020B0000AC0113331F0183709F47CC0103331F005
:1020C00002C091E004C090E08FEF01C090E0209149
:1020D0008901292720938901482F50E04B3351056E
:1020E00008F064C0FA01EC5CFF4F0C94F51D90936E
:1020F0008A015DC020918A01921359C057C099236B
:1021000009F454C054C09093890110928D01992311
:1021100009F44DC0E82FF0E0E45AFE4F20918D0104
:102120009081920F90938D0142C0909389011092FB
:102130008C019923E1F1E82FF0E0EC5AFE4F209159
:102140008C019081920F90938C0131C09093890102
:1021500010923901992359F1E82FF0E0E35BFE4F2B
:10216000209139019081920F9093390120C01092F3
:1021700038019923E1F0E82FF0E0EC5BFE4F20916D
:1021800038019081920F9093380111C010928B0109
:10219000992369F0E82FF0E0E15CFE4F20918B017C
:1021A0009081920F90938B0102C021118FEF8F5F6E
:1021B00080933E0184E391E00E942E19882309F464
:1021C000E7C080913F01909140010E9708F4E0C074
:1021D00087E0E3E6F1E0DE01119601900D928A9529
:1021E000E1F787E0FE013196DE011F9601900D9226
:1021F0008A95E1F718861092980161E0CE01089661
:102200000E94610C882309F4BBC084EA8093BC005F
:1022100014E68091BC0087FD07C0112309F458C063
:102220000E943A0C1150F5CF112309F451C080914E
:10223000B900887F883009F04BC081ED8093BB00E6
:1022400084E88093BC0014E68091BC0087FD06C042
:102250001123F1F10E943A0C1150F6CF1123C1F174
:102260008091B900887F803499F5CE0108967C0171
:1022700010E044E8C42E54ECB52E163021F0B09294
:10228000BC0000E503C0C092BC0008E534E6D32ED4
:102290008091BC0087FD06C0DD20B9F00E943A0C99
:1022A000DA94F6CFDD2089F08091B900887F90E044
:1022B000202F30E08217930741F48091BB00F70193
:1022C00081937F011F5F1730C1F681E0173009F05D
:1022D00080E094E99093BC00E9E4F0E031970000DD
:1022E000E9F71092BC00882309F44AC081E080938A
:1022F0009801888587FD44C0982F92959F708F70B4
:10230000FAE09F9F800D1124898B8985982F9295E3
:102310009F708F702AE0929F800D1124888B8A8590
:10232000982F92959F708F703AE0939F800D1124A3
:102330008F878C85982F92959F708F70EAE09E9F73
:10234000800D11248A8B8D85982F92959F708F70A8
:10235000FAE09F9F800D11248B8B2E85822F829512
:102360008F703AE0839FC00111248053984F2F70E3
:10237000820F911D9D8B8C8BCE010F960E941D1597
:1023800080919801882321F0CE010F960E94440C81
:1023900080E391E00E942E198823B9F180E48093B4
:1023A0007C0080917A00806480937A0080917A002A
:1023B00086FDFCCF2091780080917900837030E019
:1023C000382B8FEF93E0821B930B9595879595950E
:1023D0008795853091051CF410929A0116C0893CAE
:1023E000910524F084E680939A010FC09C0125504A
:1023F000310944E6429FC001439F900D112463ECD4
:1024000070E00E94E11D60939A01A8950E94E70E7A
:10241000807892708038910511F45F9A01C05F98BE
:1024200065960FB6F894DEBF0FBECDBFDF91CF919A
:102430001F910F91FF90EF90DF90CF90BF90089584
:10244000F89498E088E10FB6F894A895809360001E
:102450000FBE90936000FFCFFC018081840F8083CA
:1024600080E09081961750F047FF04C0960F90834C
:102470008150F7CF961B90838F5FF3CF0895FC01B7
:102480008081883150F481818C3338F491E08281ED
:102490008C3308F090E0892F01C080E081700895AE
:1024A000DC01FB019C9180819817B0F0891790F0B6
:1024B00011969C9111978181981770F0891750F0AF
:1024C00012962C919281291738F081E0921728F00A
:1024D00080E0089581E008958FEF0895DC01FB010D
:1024E00012962D913C911397828193812817390779
:1024F000B0F08217930788F011969C911197818113
:10250000981768F0891748F02C919081291738F0B6
:1025100081E0921728F080E0089581E008958FEF20
:1025200008959C0183709927892B81F4C90164E681
:1025300070E00E94CD1D892B59F4C90160E971E05A
:102540000E94CD1D9C0181E0232B19F080E00895AD
:1025500081E00895CF93DF93FC0182819381860F00
:10256000911D67FD9A95893223E2920718F088E25F
:1025700093E206C0843A26E0920710F484EA96E0DB
:10258000938382838181823061F480818D3149F42B
:10259000EF01828193810E949112811102C08CE12E
:1025A0008883DF91CF910895823039F4CB010E9466
:1025B0009112882341F08DE108958D7F843029F0B8
:1025C000893029F402C08CE108958EE108958FE1ED
:1025D0000895CF93FC0162817381CB01845A9640A8
:1025E00085389C4168F481819FEF980F9C3040F4BE
:1025F000C081CC2329F00E94D41291E08C1708F4FA
:1026000090E0892FCF910895CF93DF93EC01462F6F
:102610008981815089836CE0CE0101960E942C1241
:1026200099819F5F9983682FCE010E94AA126A81C7
:102630007B8189810E94D4129881891708F488834C
:10264000DF91CF910895FF920F931F93CF93DF9364
:10265000EC01162F6A817B8189810E94D412F82EA9
:10266000012F10166CF48881F81206C061E0CE01CB
:102670000E94041381E001C08F5F88830150F1CF75
:10268000812F17FD80E0181B112369F088818130AC
:1026900031F46FEFCE010E940413F88202C0815022
:1026A00088831F5FF1CFDF91CF911F910F91FF9032
:1026B0000895CF93DF93DC011296CD91DC911397AF
:1026C0001196EC911197E33008F42197F0E0E95B63
:1026D000FC4FE4918C919E01280F311DCE019695FF
:1026E000879596958795280F391FCE0160E971E08F
:1026F0000E94CD1D260F371F2E0F311DCE0164E61F
:1027000070E00E94CD1DC901861B970B67E070E049
:102710000E94CD1D009711F487E090E0DF91CF91EA
:102720000895EF92FF920F931F93CF937C01FC01CA
:10273000C181C150008110E0CC2351F0F7016281CA
:1027400073818C2F0E94D412080F111DC150F4CF39
:10275000C801CF911F910F91FF90EF9008958F9234
:102760009F92AF92BF92CF92DF92EF92FF920F9320
:102770001F93CF93DF9300D000D0CDB7DEB78C018D
:10278000FC01C280D380F8E9CF16F8E0DF0608F03C
:102790003AC10E9491137C01E11480E8F80609F423
:1027A0003AC1C6018C56974063E170E00E94CD1D8E
:1027B0009C0167E0862E912CC60189569740B40192
:1027C0000E94CD1D5C019C2D9370E92FF0E0AA0CB6
:1027D000BB1CAA0CBB1C43E1429FC001439F900D50
:1027E000112448966EE170E00E94E11DDC01482F43
:1027F00084E3C81688E0D80678F4CF01880F991FC3
:102800008A0D9B1D56E05A9FB0015B9F700D1124ED
:10281000860F971F05960EC0CF01880F991F8A0D4E
:102820009B1D56E05A9FB0015B9F700D1124860FCF
:10283000971F0696B4010E94E11D642F70E06A5E46
:102840007F4F680F711D840F6032710524F48A5E1A
:10285000898383E00FC0895089838A3111F483E131
:1028600007C0893131F44C3121F42B3010F082E172
:10287000898384E08A83DC82CB82CE0101960E9428
:102880009113B82E88E189838CE08A83DC82CB8225
:10289000CE0101960E94591336E1873009F0381BAA
:1028A000F8012181213039F48081813009F481C01F
:1028B000863009F480C08B2D90E0AC01445351095F
:1028C000E416F50609F479C04C5F5F4FE416F5068F
:1028D00009F475C04F5F5F4FE416F50609F471C047
:1028E0004F5F5F4FE416F50609F46DC0455D5F4F1D
:1028F000E416F50609F469C04F5F5F4FE416F5066C
:1029000009F465C0E816F90609F463C04D5F5F4F2E
:10291000E416F50609F45FC0253029F4F80140817A
:10292000413009F45AC0AC01495D5F4FE416F50629
:1029300009F455C0465F5F4FE416F50609F451C02F
:102940004F5F5F4FE416F50609F44DC0CC96E816CC
:10295000F90609F44AC0283039F4F80180818F3033
:1029600009F051C081E158C02A3049F4F801808152
:102970008330E9F18F3109F046C083E14DC02B303F
:1029800041F4F80180818130A1F138133CC085E128
:1029900043C02C30C1F5F8018081863061F1883167
:1029A00061F1893161F18A3161F18F3161F58AE13B
:1029B00033C082E031C083E02FC084E02DC085E0C9
:1029C0002BC086E029C087E027C088E025C089E0C9
:1029D00023C08AE021C08BE01FC08CE01DC08DE0C9
:1029E0001BC08EE019C08FE017C080E115C082E1E6
:1029F00013C084E111C086E10FC087E10DC088E1FA
:102A00000BC089E109C0C8010E9459139AEF980FC1
:102A100081E0923008F080E00F900F900F900F90BF
:102A2000DF91CF911F910F91FF90EF90DF90CF90AA
:102A3000BF90AF909F908F900895CF93DF93EC015C
:102A40000E943F12882329F0CE0103960E94E912CA
:102A500002C080E090E08170DF91CF910895CF9324
:102A6000DF93EC01462F68E10E942C12682FCE0103
:102A70000396DF91CF910C942313CF93DF93EC0156
:102A8000462F6CE301960E942C12682FCE01DF9135
:102A9000CF910C942F15CF93DF93EC01462F6CE36D
:102AA00002960E942C12682FCE01DF91CF910C94D8
:102AB0003D1503960C9423130F931F93CF93DF932D
:102AC000EC018B016D5F7F4F03960E946E128111A6
:102AD00008C0B801CE01DF91CF911F910F910C94E6
:102AE0005012DF91CF911F910F910895CF93DF93F3
:102AF000EC019C8194509630D0F0CE0103960E9458
:102B00005913873009F480E09C81933091F42B8134
:102B1000293128F130E0281B310929313105FCF039
:102B2000811105C088818230D0F08230B1F081E01F
:102B300017C09A30A1F42B812931C8F330E0281B4B
:102B40003109293131059CF3811109C08881823016
:102B500070F3823021F483E003C082E001C080E0A2
:102B6000DF91CF9108951F93CF93DF93162FEA0142
:102B7000682FCA010E942F15112369F0CE010E940F
:102B800076158150823038F461E0CE01DF91CF912B
:102B90001F910C942F15DF91CF911F9108950F93E2
:102BA0001F93CF93C82F8A01662339F0CA010E9470
:102BB00076158D7F813009F4CF5F6C2F6195C80148
:102BC000CF911F910F910C942F159091B3019817ED
:102BD00029F08093B30181E08093A701089590913B
:102BE0005301981769F087FF03C01092530105C085
:102BF00080310CF08FE08093530181E08093A70136
:102C00000895809153010895E82FF0E0E855FE4FB4
:102C10008081462F50E0282F2F7730E0421753074E
:102C200051F08078682B60838091B301882319F07C
:102C300081E08093A7010895E82FF0E0E855FE4F6A
:102C40008081982F991F9927991F961749F066231D
:102C500011F0806801C08F77808381E08093A701A5
:102C60000895CF93C0E060E08C2F0E940416CF5FE0
:102C7000C830C9F7CF9108950F931F93CF938C015C
:102C8000C0E0D801ED918D01EE2391F080EE8E0F22
:102C9000863538F40E2E000CFF0BE45BFC4F64917C
:102CA00001C069E48C2F0E940416CF5FC83049F739
:102CB000CF911F910F9108950F931F93CF93DF939F
:102CC000EC0100E010E0802FFE01E00FF11FE49125
:102CD000EE2399F090EE9E0F963538F40E2E000CF0
:102CE000FF0BE45BFC4F649101C069E40E94041691
:102CF0000F5F1F4F0830110531F7DF91CF911F9102
:102D00000F9108958CE08093520181E08093A70198
:102D10000895809152010895CF939091B101981731
:102D200059F08093B101C1E0C093B0018AE491E011
:102D30000E94FD18C093A701CF91089581E00C94E3
:102D4000E515EF92FF920F931F93CF93809152015D
:102D50008C3009F435C08EE491E00E942619882356
:102D600009F444C0E0915201F0E0EE0FFF1FEC5A6D
:102D7000FC4F259134919091B20183E0989F200DF2
:102D8000311D1124F9018491319664913196C491D9
:102D90008F3F19F40E94821629C09F5F9093B20161
:102DA0008D3F19F40E94311602C00E940416FAE009
:102DB000CF9FB00111248EE491E00E94ED18CBCF9B
:102DC0008091B301882391F08091B101882371F043
:102DD0008AE491E00E942E19882341F08091B0018D
:102DE00091E089278093B0019093A7018091A7017A
:102DF000882309F447C01092A70160E089E00E948F
:102E00000D0F609153018AE00E940D0F67E08BE087
:102E10000E940D0F61E08CE00E940D0F60E08FE0DA
:102E20000E940D0F08EA11E087E0E82EF12CC0E0C7
:102E30008091B301882391F08091B10190E00E2C34
:102E400002C0959587950A94E2F780FF04C08091AF
:102E5000B001882319F0F801608109C08DEF8C0F53
:102E6000823020F4F8016081607801C060E0CF5FBB
:102E70008C2F0E940D0F0F5F1F4FF1E0EF1AF1082A
:102E8000C830B1F6CF911F910F91FF90EF90089548
:102E9000CF9380935201C1E0C093A7018C3059F0C9
:102EA0001092B2018EE491E00E94FD18C093B0012F
:102EB000CF910C94A116CF91089580E00C94E51564
:102EC0000E949C0F0E94391C0E949E160E941D09A0
:102ED0000E94EC0F882349F00E94EF0F0E94911C82
:102EE0000E94A1160E944109F3CF0E94390C0E9452
:102EF0005D170E94301D0C9420121092B50180E0E5
:102F00000E948C1688E00E94481784E00E94FB1BF8
:102F100087E591E00E94D21843E050E064E571E05B
:102F200085E090E00C94091CFF920F931F93CF93C0
:102F3000DF93CDB7DEB72A970FB6F894DEBF0FBE8A
:102F4000CDBF8091B501882319F08130F1F147C0E0
:102F50008E010F5F1F4F8AE0F80111928A95E9F701
:102F600066E579E0C8010E945D1D809154018831B9
:102F700018F5909155019C33F8F48A3020F460E202
:102F8000C8010E943D1D6091540170E0C8010E947B
:102F9000711D6DE2C8010E943D1D809155018A306E
:102FA00020F460E3C8010E943D1D6091550170E06E
:102FB000C8010E94711D05C065E379E0C8010E9447
:102FC0005D1DC8010E943C160EC00E94B9068823F0
:102FD00019F08DE499E005C084E499E002C08BE328
:102FE00099E00E945C160E94CE08882309F44BC029
:102FF0008091B4018823C9F01092560143E050E05B
:1030000064E571E085E090E00E940C1C81E00E9484
:10301000B00688E00E94FB1B81E00E94481780E018
:103020000E948C161092B4012BC08091B5018823A8
:1030300019F0813059F01EC081E08093B40184EC16
:103040000E948C1684E00E94FB1B1DC00E94B906E2
:10305000882341F080E00E94B00689E00E94FB1BBB
:1030600082E00CC081E00E94B00688E00E94FB1B59
:1030700081E004C085E00E94FB1B89E00E944817A4
:1030800081E00E94CB080E94D108182F81110AC04C
:103090000E94D408882309F46AC087E591E00E9461
:1030A000D21865C08091B401012F882309F44AC069
:1030B0001016CCF483E00E94FB1B809155018B5FBE
:1030C000883318F4809355010CC0109255018091FB
:1030D00054018F5F883118F48093540102C010921C
:1030E00054010150E5CF812F17FD80E0181B0CE340
:1030F00088E1F82E112361F283E00E94FB1B80918E
:103100005501853068F480915401811102C0F0921C
:1031100054018091540181508093540100935501D2
:10312000809155018550809355011F5FE3CF8091B9
:10313000B501823031F08F5F8093B50183E00E944A
:10314000FB1B015010169CF3812F17FD80E0181B0C
:10315000112309F49DCF8091B501882331F081506E
:103160008093B50183E00E94FB1B1F5FF1CF87E5D1
:1031700091E00E942619882349F085E00E94FB1BFC
:1031800089E00E94481781E00E94CB082A960FB67A
:10319000F894DEBF0FBECDBFDF91CF911F910F918D
:1031A000FF900895CF93DF93EC0188812981922FBE
:1031B0009F7321E0892B09F020E0898120FB87F9AA
:1031C000898386FD03C00E94E70E02C00E94F50EAF
:1031D0009B838A83DF91CF91089569392AE372072F
:1031E00010F068E97AE3FC016083372F3F73218197
:1031F000207C232B21830C94D218FC012181206890
:1032000021830895CF93DF93EC01998197FD19C035
:1032100096FD03C00E94E70E02C00E94F50E2A81AF
:103220003B81AC01421B530B28818981382F3F73AE
:103230004217530720F4C901841B950B04C0806812
:10324000898380E090E0DF91CF9108950E94021978
:1032500021E0892B09F020E0822F08950F931F931E
:10326000CF938C010E942619C82F882319F0C8011A
:103270000E94D2188C2FCF911F910F910895462F45
:1032800050E04D30510560F5FA01E159FF4F0C94C3
:10329000F51D6CE27AE026C065E27AE023C062E2C6
:1032A0007AE020C06DE17AE01DC06AE17AE01AC0E0
:1032B00065E17AE017C06EE07AE014C068E07AE079
:1032C00011C063E07AE00EC06EEF79E00BC06AEFE8
:1032D00079E008C064EF79E005C06EEE79E002C0E5
:1032E0006BEE79E00C945D1DAF92BF92CF92DF92AE
:1032F000EF92FF920F931F93CF93DF93CDB7DEB77B
:103300002A970FB6F894DEBF0FBECDBF6C015B01EC
:103310007A018E010F5F1F4F8AE0F80111928A95A2
:10332000E9F7BA01C8010E945D1DC8010E943A1D5B
:103330008F5F8A9DB0018B9D700D11246E0D7F1DD6
:10334000C6010E945D1D2A960FB6F894DEBF0FBE1F
:10335000CDBFDF91CF911F910F91FF90EF90DF9044
:10336000CF90BF90AF900895CF92DF92EF92FF92EF
:103370000F931F93CF93DF937C016B010E94CE08C4
:10338000811147C0E114F10429F4D1E081E0C816AD
:10339000D10409F0D0E000915B0110915C010E9422
:1033A000D108C82F882379F1D0FD0BC0D82F19C0C0
:1033B000860183E00E94FB1B1C1644F4C150CC2301
:1033C00011F1E016F106A1F38701F3CFCF5FF7CF3C
:1033D0000C151D052CF40F5F1F4F83E00E94FB1B93
:1033E000D1501D16ACF38C2FC7FD80E0C81BCC2339
:1033F00051F0E016F1062CF40150110983E00E940F
:10340000FB1BCF5FF4CF10935C0100935B0181E065
:1034100001C080E0DF91CF911F910F91FF90EF905D
:10342000DF90CF900895CF93DF931F92CDB7DEB793
:103430001092B7011092B60141E050E0BE016F5FFB
:103440007F4F80E090E00E94091C898190E090937A
:103450005C0180935B018AE00E94481780E00E9433
:103460008C168FE00E94FB1B8DE591E00E94D21824
:103470000F90DF91CF9108950F931F93CF93DF9318
:10348000CDB7DEB765970FB6F894DEBF0FBECDBFE0
:103490008E01055F1F4F8AE0F80111928A95E9F7C6
:1034A0006091B701C8010E943F1960E2C8010E9403
:1034B0003D1D60915B0170915C01E091B7018E2F21
:1034C00090E08D309105D8F4FC01E458FF4F0C9446
:1034D000F51D41EC59E00FC045EB59E00CC0C801A7
:1034E0000E94711D11C04DE659E005C04DEA59E03A
:1034F00002C047E659E0C8010E94741905C063E69E
:1035000079E0C8010E945D1DC8010E943A1D883003
:1035100028F460E2C8010E943D1DF6CFC8010E9458
:103520003C168091B601882309F4ACC0E091B70144
:103530008E2F90E08D309105F0F4FC01E757FF4F9E
:103540000C94F51D66E070E010C060EF70E005C0FF
:1035500069E070E002C063E670E081E090E007C0DF
:103560006FE070E002C061E070E080E090E00E94F7
:10357000B41981111BC1E091B70120915B012D8B22
:103580008E2F90E08D30910508F075C0FC01EA5651
:10359000FF4F0C94F51D41E050E0BE016B5E7F4F84
:1035A00080E090E007C041E050E0BE016B5E7F4FDD
:1035B00081E090E00E940C1C5EC041E050E0BE0142
:1035C0006B5E7F4F83E090E0F5CF41E050E0BE01BD
:1035D0006B5E7F4F84E090E0EDCF41E050E0BE01B4
:1035E0006B5E7F4F88E090E0E5CF41E050E0BE01A8
:1035F0006B5E7F4F89E090E0DDCF41E050E0BE019F
:103600006B5E7F4F8AE090E0D5CF41E050E0BE0195
:103610006B5E7F4F8BE090E0CDCF41E050E0BE018C
:103620006B5E7F4F8CE090E0C5CF41E050E0BE0183
:103630006B5E7F4F8DE090E0BDCF41E050E0BE017A
:103640006B5E7F4F8EE090E0B5CF213011F40E9489
:10365000141C8D89813079F487E0EAE6F1E0DE011F
:10366000119601900D928A95E1F7CE0101960E9484
:10367000340F0E94E40E1092B60182E10E94FB1BFF
:1036800080E030C00E94CE08882379F18091B70194
:103690008D3069F480E00E948C168BE00E94481700
:1036A00080E10E94FB1B81E00E94CB087FC081E18A
:1036B0000E94FB1B81E08093B6016091B7018E01EF
:1036C0000F5F1F4F8AE0F80111928A95E9F7C80150
:1036D0000E943F19C8010E943A1DE82FF0E0E65A07
:1036E000F64F84910E948C1661C00E94D108182F59
:1036F000882309F45BC0082F101664F48091B70189
:103700008D3031F08F5F8093B70183E00E94FB1B07
:103710000150F2CF812F17FD80E0181BE091B70117
:10372000112359F0EE2339F08FEF8E0F8093B701FC
:1037300083E00E94FB1B1F5FF1CF8E2F90E08B3048
:10374000910568F5FC01ED55FF4F41E050E0BE01E9
:103750006F5F7F4F0C94F51D80E090E002C081E028
:1037600090E00E94091C1CC083E090E0FACF84E046
:1037700090E0F7CF88E090E0F4CF89E090E0F1CFDF
:103780008AE090E0EECF8BE090E0EBCF8CE090E031
:10379000E8CF8DE090E0E5CF8EE090E0E2CF1982B7
:1037A000898190E090935C0180935B010E94D40832
:1037B000882321F08DE591E00E94D2188DE591E0FB
:1037C0000E942619882361F080E00E948C168BE00D
:1037D0000E94481780E10E94FB1B81E00E94CB08F9
:1037E00065960FB6F894DEBF0FBECDBFDF91CF91C7
:1037F0001F910F910895833111F40C94240FE82F39
:10380000F0E0EE0FFF1FEE5CF54F859194910C9464
:10381000180F0A960C94030F0A960E94080F109234
:1038200062011092610108950F931F93CF93DF936C
:103830001F92CDB7DEB70AE010E0F801E65DF44F65
:10384000E491E98341E050E0BE016F5F7F4FC80122
:103850000E94080F0F5F1F4F0931110571F7109279
:103860006201109261010F90DF91CF911F910F9132
:103870000895EF92FF920F931F93CF93DF9300D0A1
:10388000CDB7DEB72AE0E22EF12C0FEF1FEF41E0BB
:1038900050E0BE016F5F7F4FC7010E94030F898117
:1038A000082788E0A801569547959801217033278D
:1038B00000FF02C028E034E88A0102271327815064
:1038C00089F72FEFE21AF20A89E1E816F104F9F616
:1038D0000F3F2FEF120711F400E010E042E050E03C
:1038E000BE016F5F7F4FC7010E94030F89819A81DC
:1038F00025E2E216F10439F022E0E20EF11C8F3FDE
:103900002FEF920759F38017910711F00E94141CB2
:103910000F900F90DF91CF911F910F91FF90EF903B
:103920000895EF92FF921F93CF93DF9300D000D0C2
:103930001F92CDB7DEB780916101909162018F3FF8
:103940002FEF920709F481C041E050E0BE016B5FA8
:103950007F4F0A960E94030F20916101309162010E
:103960002115310531F48FEF9FEF9093B9018093CA
:10397000B8014D818091B8019091B901842748E048
:10398000FC01F695E795BC016170772780FF02C0C6
:1039900068E074E8CF0186279727415089F7909314
:1039A000B9018093B8012F5F3F4F2F30310529F0C7
:1039B000309362012093610148C02FEF3FEF3093B5
:1039C0006201209361018F3F2FEF920719F09C83D2
:1039D0008B8302C01C821B8210E039E1E32EF12CA4
:1039E00042E050E0BE016F5F7F4FC7010E94030FAE
:1039F00089819A818F3F2FEF920731F422E0E20E06
:103A0000F11C1F5F173061F72B813C8182179307F0
:103A1000E1F08FEF9FEF9A83898342E050E0BE018F
:103A20006F5F7F4FC7010E94080F1F5F173008F0BC
:103A300010E0812F90E0880F991F42E050E0BE0116
:103A40006D5F7F4F49960E94080F0F900F900F9067
:103A50000F900F90DF91CF911F91FF90EF900895FD
:103A60008091610190916201019619F00E94911C70
:103A7000F7CF0895FC0181850895FC012185283048
:103A800048F4E20FF11D60832F5FFC012187E20FF4
:103A9000F11D108208950F931F93CF93DF938C0134
:103AA000EB016991662321F0C8010E943D1DF9CF09
:103AB000DF91CF911F910F9108950F931F93CF9393
:103AC000DF938C01EB01FE016491662329F0C801AC
:103AD0000E943D1D2196F7CFDF91CF911F910F914D
:103AE0000895CF92DF92EF92FF920F931F93CF939F
:103AF000DF937C018B0177FF17C06DE20E943D1DB3
:103B0000011580E8180769F469E771E0C701DF91E2
:103B1000CF911F910F91FF90EF90DF90CF900C9479
:103B20004B1D119501951109C0E1D7E220E08AE013
:103B3000C82ED12CC801BE010E94CD1DCB01B601FB
:103B40000E94CD1D211102C0009731F060E3680F83
:103B5000C7010E943D1D21E0CE01B6010E94CD1D8E
:103B6000EB016130710511F421E0E4CF209711F7EA
:103B7000DF91CF911F910F91FF90EF90DF90CF9049
:103B80000895991B79E004C0991F961708F0961BB9
:103B9000881F7A95C9F780950895AA1BBB1B51E130
:103BA00007C0AA1FBB1FA617B70710F0A61BB70BAD
:103BB000881F991F5A95A9F780959095BC01CD0152
:103BC000089597FB072E16F4009407D077FD09D0CF
:103BD0000E94CD1D07FC05D03EF4909581959F4F26
:103BE0000895709561957F4F0895EE0FFF1F059022
:103BF000F491E02D0994DC01CB01FC01F999FECF91
:103C000006C0F2BDE1BDF89A319600B40D92415064
:103C10005040B8F70895DC01A40FB51F4150504043
:103C200048F0CB01840F951F2E910E941C1E41501D
:103C30005040D0F70895262FF999FECF92BD81BD4F
:103C4000F89A019700B4021639F01FBA20BD0FB6DA
:0E3C5000F894FA9AF99A0FBE0895F894FFCFEF
:103C5E0000C000003280000000C000000000000123
:103C6E0001D007020F80000001DC85000000C000BB
:103C7E00003280000096800000FF64800000010189
:103C8E002C810000B8CB000001013CC00000006098
:103C9E00EA01FFFFFFFFFFFFFF782C81000000808D
:103CAE0000000C0F0700000AC00000008098BA0048
:103CBE0000FFFFFFFFFFFFFFFFFFFFFFFFFFFFFF05
:103CCE00FF010204080A1428503332373638000038
:00000001FF
